:020000040000FA
:06000000C93001303A286E
:08000800A000030EA100831209
:100010008B1C32288B1031181428B11C3228643004
:10002000010203183128182800001628172818285C
:1000300019281A281B281C281D281E281F283110A3
:10004000B114A810031005190314AA0DA90DA80DC9
:10005000B00B322831152A08AF002908AE00280855
:10006000AD00B11081010B11210E8300A00E200EF6
:02007000090085
:0C007400203084008001840A80300402E7
:10008000031C3C281230B000F02183160C3085058B
:1000900087018312850187010730990000309A009B
:1000A000103083168E008312603083168F00831207
:1000B0000030831691009F008312C83083168100A0
:1000C000831231309000003083168C008312103080
:1000D0008B00831600309B001C141A088312BC008E
:1000E000851DE222831610309B001C141A0883120F
:1000F000BD00831630309B001C141A088312DE00EA
:10010000C92281018E018F010B118B100B108C0104
:100110008B1798203119AE20B30B96280310851940
:100120000314B90DF030390203195421282389280A
:100130006400311808000B1D08000B11B1103114B8
:100140001230B000051DA928321483160113831242
:100150000800321083160117831208003111013094
:10016000B7008B132030370783169B001C141A0826
:100170008312A400A500C030A506103037078316EF
:100180009B001C141A088312A30000303707831643
:100190009B001C141A088312A2008B17321CD6284D
:1001A00022090339A200A309A409A50922082D02E6
:1001B000031D4E2923082E02031D4E2924082F0259
:1001C000031D4E2901303702031DEB283D18EB2893
:1001D0003D143E14FD2102303702031DF428BD18E2
:1001E000F428BD143E140C2203303702031DFD28F1
:1001F0003D19FD283D153E14182204303702031D19
:100200000629BD190629BD153E14242205303702E2
:10021000031D0F293D1A0F293D163E1433220630C7
:100220003702031D1829BD1A1829BD163E143F2296
:1002300007303702031D21293D1B21293D173E149C
:100240004B2208303702031D2A29BD1B2A29BD175E
:100250003E14562209303702031D33295E18332914
:100260005E143E1461220A303702031D3C29DE1859
:100270003C29DE143E146C220B303702031D452945
:100280005E1945295E153E1477220C303702031D96
:100290004E29DE194E29DE153E148222B70A0D3092
:1002A000370203180800B1280130B600B300B400CB
:1002B000B500B70085018701B1139820B30B9C29C5
:1002C000031085190314B90DF03039020319C3293D
:1002D000B40B9C290130370203198D2202303702FA
:1002E0000319922203303702031997220430370290
:1002F00003199C22053037020319A1220630370268
:100300000319A622073037020319AB22083037023F
:100310000319B022093037020319B5220A30370217
:100320000319BA220B3037020319BF220C303702EF
:100330000319C4229630B400311D5D293111321CDD
:10034000A6292D090339AD00AE09AF092F1CB11341
:100350002F1C5D29B11B5D292E185D29B1178B1348
:1003600020303707BB002F08BA00DB2110303707D9
:10037000BB002E08BA00DB2100303707BB002D0878
:10038000BA00DB218B1785018701B70AB6010D3052
:100390003702031C5D29C92208003E1C08003E10DC
:1003A0001030BB003D08BA00DB213030BB005E08D6
:1003B000BA00DB2108008B133A0883161C159A003B
:1003C00083123B0883169B0055309D00AA309D0088
:1003D0009C1464009C18E9291C1183128B170800D7
:1003E000FF30C800CA15CB15CC15CD15CE15CF15CD
:1003F000D015D115D215D3150800C130BD05FF3079
:10040000DE050130C405C0000030C200C600BC18C3
:100410005F14BC18DF140800C230BD05FF30DE05D4
:100420000230C405C0000030C200C6005F100800E2
:10043000C430BD05FF30DE050630C405C000003005
:10044000C200C6005F100800C830BD05FF30DE05E1
:100450001830C405C0000030C200C600BC185F14CC
:10046000BC18DF140800D030BD05FF30DE05223097
:10047000C405C0000030C200C6005F100800E030B4
:10048000BD05FF30DE052630C405C0000030C200C7
:10049000C6005F1008007F30BD05C030DE05C030EB
:1004A000C505C1000030C300C7000800BF30BD054E
:1004B000C030DE053030C505C1000030C300C700C4
:1004C00008003F30BD05C130DE059030C505C100D4
:1004D0000030C300C70008003F30BD05C230DE0554
:1004E000C030C505C1000030C300C70008003F3060
:1004F000BD05C430DE053030C505C1000030C30085
:10050000C70008003F30BD05C830DE059030C50586
:10051000C1000030C300C70008001030850600305D
:100520008706080020308506003087060800213045
:1005300085060030870608000230850602308706EF
:100540000800203085060430870608002130850623
:10055000043087060800003085061830870608003A
:1005600000308506213087060800003085060930F6
:10057000870608000030850618308706080000301E
:100580008506213087060800003085060930870679
:1005900008003D18FD21BD180C223D191822BD1977
:1005A00024223D1A3322BD1A3F223D1B4B22BD1B84
:1005B00056225E186122DE186C225E197722DE193F
:1005C00082220800B601B301B4013C1CEA2ABC0136
:1005D000BC14EC2ABC013C143C08B6006400F02AB0
:1005E000F12AF22AF32AF42AFF30B41B8500B41F43
:1005F0008501B30BEE2AB40BEE2A0310B60CB60835
:10060000031DEE2A0030BB003C08BA00DB210800C5
:1006100005125C180516DC1C8512DC1885165C1D9D
:1006200005105C190514DC1D8510DC1985145C1E91
:1006300087105C1A8714DC1E0711DC1A07155C1F73
:1006400007105C1B0714DC1F8712DC1B87160800D1
:100650008F08031908008F0178308E00C80F5A2DBB
:10066000C80A441C582B461C492BCA1C3A2BCA01E9
:100670004A15662B4A1D3F2BCA01CA15662BCA1D97
:10068000442BCA014A16662B4A1E662BCA01CA149D
:10069000662B4A1D4E2BCA014A16662BCA1D532BC8
:1006A000CA014A16662B4A1E662BCA01CA14662B5B
:1006B000CA1C5D2BCA014A15662B4A1D622BCA0152
:1006C000CA15662B4A1E662BCA014A15C41C8D2BFF
:1006D000C61C7E2BCB1C6F2BCB014B159B2B4B1DB4
:1006E000742BCB01CB159B2BCB1D792BCB014B1640
:1006F0009B2B4B1E9B2BCB01CB149B2B4B1D832B7E
:10070000CB014B169B2BCB1D882BCB014B169B2B68
:100710004B1E9B2BCB01CB149B2BCB1C922BCB01C9
:100720004B159B2B4B1D972BCB01CB159B2B4B1E9E
:100730009B2BCB014B15441DC22B461DB32BCC1C50
:10074000A42BCC014C15D02B4C1DA92BCC01CC15C6
:10075000D02BCC1DAE2BCC014C16D02B4C1ED02B4D
:10076000CC01CC14D02B4C1DB82BCC014C16D02B6B
:10077000CC1DBD2BCC014C16D02B4C1ED02BCC014C
:10078000CC14D02BCC1CC72BCC014C15D02B4C1D22
:10079000CC2BCC01CC15D02B4C1ED02BCC014C1526
:1007A000C41DF82BC61DE92BCD1CDA2BCD014D1530
:1007B0005F13062C4D1DDF2BCD01CD15062CCD1D55
:1007C000E42BCD014D16062C4D1E062CCD01CD146B
:1007D000062C4D1DEE2BCD014D16062CCD1DF32BF9
:1007E000CD014D16062C4D1E062CCD01CD14062C28
:1007F000CD1CFD2BCD014D15062C4D1D022CCD0120
:10080000CD15062C4D1E062CCD014D155F1B2F2C32
:10081000441E2F2C461E202CCE1C112CCE014E1512
:100820003D2C4E1D162CCE01CE153D2CCE1D1B2C65
:10083000CE014E163D2C4E1E3D2CCE01CE143D2C2D
:100840004E1D252CCE014E163D2CCE1D2A2CCE0140
:100850004E163D2C4E1E3D2CCE01CE143D2CCE1CF2
:10086000342CCE014E153D2C4E1D392CCE01CE150B
:100870003D2C4E1E3D2CCE014E15C41E642CC61EB2
:10088000552CCF1C462CCF014F15722C4F1D4B2CD5
:10089000CF01CF15722CCF1D502CCF014F16722CCB
:1008A0004F1E722CCF01CF14722C4F1D5A2CCF012A
:1008B0004F16722CCF1D5F2CCF014F16722C4F1E7E
:1008C000722CCF01CF14722CCF1C692CCF014F1585
:1008D000722C4F1D6E2CCF01CF15722C4F1E722C17
:1008E000CF014F15DF189B2C451E9B2C471E8C2CCF
:1008F000D01C7D2CD0015015A92C501D822CD0016C
:10090000D015A92CD01D872CD0015016A92C501E13
:10091000A92CD001D014A92C501D912CD001501617
:10092000A92CD01D962CD0015016A92C501EA92CF4
:10093000D001D014A92CD01CA02CD0015015A92C6A
:10094000501DA52CD001D015A92C501EA92CD001CA
:100950005015DF18D22CC51ED22CC71EC32CD11C9B
:10096000B42CD1015115E02C511DB92CD101D11558
:10097000E02CD11DBE2CD1015116E02C511EE02CD3
:10098000D101D114E02C511DC82CD1015116E02CFD
:10099000D11DCD2CD1015116E02C511EE02CD101DE
:1009A000D114E02CD11CD72CD1015115E02C511DB4
:1009B000DC2CD101D115E02C511EE02CD1015115B8
:1009C000DF180A2D451F0A2D471FFB2CD21CEC2CCB
:1009D000D2015215DF13182D521DF12CD201D21560
:1009E000182DD21DF62CD2015216182D521E182D7C
:1009F000D201D214182D521D002DD2015216182DDD
:100A0000D21D052DD2015216182D521E182DD201BD
:100A1000D214182DD21C0F2DD2015215182D521D93
:100A2000142DD201D215182D521E182DD201521597
:100A3000DF18432DDF1B432DC51F432DC71F342D4A
:100A4000D31C252DD3015315512D531D2A2DD30110
:100A5000D315512DD31D2F2DD3015316512D531EB8
:100A6000512DD301D314512D531D392DD3015316BC
:100A7000512DD31D3E2DD3015316512D531E512DF3
:100A8000D301D314512DD31C482DD3015315512D0F
:100A9000531D4D2DD301D315512D531E512DD3016F
:100AA0005315CD214008C4004108C5005F18DF146C
:100AB0005F1CDF104808C9000C304A05031D0512F1
:100AC0000C304B05031D85120C304C05031D051021
:100AD0000C304D05031D85100C304E05031D87108D
:100AE0000C304F05031D07110C305005031D071076
:100AF0000C305105031D87120C305205031D0712DF
:100B00000C305305031D871149080E020318B42D3C
:100B100012304A05031D051612304B05031D8516BC
:100B200012304C05031D051412304D05031D8514AC
:100B300012304E05031D871412304F05031D071593
:100B400012305005031D071412305105031D87167E
:100B500012305205031D071612305305031D871569
:100B6000FF304802031908008F08031D0800982071
:100B700049080E02031CB42D18304A05031D051246
:100B800006304A05031D051618304B05031D851256
:100B900006304B05031D851618304C05031D051046
:100BA00006304C05031D051418304D05031D851036
:100BB00006304D05031D851418304E05031D8710A2
:100BC00006304E05031D871418304F05031D07110D
:100BD00006304F05031D071518305005031D07107B
:100BE00006305005031D071418305105031D8712E8
:100BF00006305105031D871618305205031D0712D4
:100C000006305205031D071618305305031D8711C2
:0A0C100006305305031D8715080088
:084000000100030003000700AA
:02400E00CC33B1
:10420000010003000300030003000200020002009B
:104210000200000000000000000003000300FF0097
:10422000020000000000000000000000000000008C
:104230000000C000C000C000C000C000C000FF00FF
:10424000FF00C300F300CF00FF00C300F300CF0066
:10425000FF00C300F300CF00FF00C300F300FF0026
:104260000100FF00FF00FF00FF00FF00FF00FF0054
:10427000FF00FF00FF00FF00FF00FF00FF00FF0046
:10428000FF00FF00FF00FF00FF00FF00FF00FF0036
:10429000FF00FF00FF00FF00FF00FF00FF00FF0026
:1042A000FF00FF00FF00FF00FF00FF00FF00FF0016
:1042B000FF00FF00FF00FF00FF00FF00FF00FF0006
:1042C000FF00FF00FF00FF00FF00FF00FF00FF00F6
:1042D000FF00FF00FF00FF00FF00FF00FF00FF00E6
:1042E000FF00FF00FF00FF00FF00FF00FF00FF00D6
:1042F000FF00FF00FF00FF00FF00FF00FF00AA001B
:00000001FF
